:100000002EC058C010C018951895189546C0189560
:100010001895189518951895189518951895189578
:100020001895189518950F931F930FB70F93839BEF
:1000300008C000E00DBD0CBD02BD0FBD02E00EBD4D
:1000400006C04CB45DB400E002BD0FBD0EBD00E0C3
:10005000802E902E0F910FBF1F910F9118950FEDCD
:100060000DBF0FE107BB08BB03EF01BB02BB07E0FD
:100070000ABB0BBB05E005BF00EC0ABF0BBF00E0ED
:1000800000BF05E003BF02E009BF2224332444245B
:10009000552488249924789429C00F931F930FB76F
:1000A0000F9311E0810E10E0911E0F910FBF1F9171
:1000B0000F9118950F931F930FB70F93829B08C052
:1000C00000E00DBD0CBD02BD0FBD02E00EBD06C0BF
:1000D0002CB43DB400E002BD0FBD0EBD00E0802E8B
:1000E000902E0F910FBF1F910F911895909AD99A4A
:1000F000C29A08E1081500E0090508F44CC014E8AC
:10010000211613E03106E0F018E9211618E0310657
:10011000B8F402EE021504E0030548F010E22116DF
:1001200013E0310620F090984BD0909A49D018E017
:10013000211617E0310620F0D99842D0D99A40D044
:1001400014E8411613E0510628F118E9411618E0A9
:10015000510600F514E1411615E0510620F0C29851
:10016000C198C098969818E0411617E0510610F013
:100170009498959804E1041505E0050520F0C29ACD
:10018000C19AC09A969A08E0041507E0050510F098
:10019000949A959AAECFC29AC19AC09A969A949A16
:1001A000959A90989198D998D8980AD0909A919ABF
:1001B000D99AD89A05D09DCF0895FEDFFDDF089526
:1001C000FCDFFBDFFADFF9DFF8DFF7DFF6DFF5DF73
:0401D000F4DF0895BB
:00000001FF
